:100000000428FF3FFF3FFF3F03138316073003130E
:1000100083169C0006309F0083128501FF308316F3
:10002000850083128601F0308316860083128701D3
:10003000831687010730BE000730BF000630C000BE
:100040000530C1000430C2000730C3000130C400D5
:100050000230C5000330C6008A1500208A110C301A
:100060008316CF008A1533218A110130E900422717
:100070007008CA000230E90042277008CB00E9018D
:1000800042277008CC0001308316CF008A15332137
:100090008A11CD01CE010530E9000530EA008A154C
:1000A00065238A1105308316C7000530C800CC309F
:1000B000C9008A156F228A1105308316C7000530E2
:1000C000C8004430C9008A156F228A110D30FC0027
:1000D000FF30FB00FF30FA00FC0B6F287628FB0B8B
:1000E00072287528FA0B72286F286C28BF30FB0025
:1000F000FF30FA00FB0B7D288028FA0B7D287A2838
:100100002B30FA00FA0B82280000000000000530B6
:10011000E9000530EA008A1565238A110530831647
:10012000C7000530C8005530C9008A156F228A11F2
:10013000AA012A08073C031CD7280830F2000C301B
:10014000F3002A08F000F1017208F00773080318A1
:10015000013FF1077008C7007108C9000A08C8000C
:100160008A152B248A11F00048088A007008CF00F5
:1001700005308316C7000530C8007008C9008A150D
:100180006F228A114130FB00FF30FA00FB0BC928B7
:10019000CC28FA0BC928C628C330FA00FA0BCE289F
:1001A00000002A08073A0319D728AA0A992801301B
:1001B000E9000B30EA008A15FA218A110530E900BE
:1001C0000530EA008A1565238A1105308316C700B9
:1001D0000530C8005530C9008A156F228A11AA015E
:1001E0002A08073C031C2E291A30F2000C30F300B9
:1001F0002A08F000F1017208F00773080318013FA4
:10020000F1077008C7007108C9000A08C8008A15FC
:100210002B248A11F00048088A007008CF000530AE
:100220008316C7000530C8007008C9008A156F2200
:100230008A114130FB00FF30FA00FB0B20292329F3
:10024000FA0B20291D29C330FA00FA0B25290000DA
:100250002A08073A03192E29AA0AF0280230E900D1
:100260000B30EA008A15FA218A110530E9000530C1
:10027000EA008A1565238A1105308316C700053008
:10028000C8005530C9008A156F228A11AA012A08B0
:10029000073C031C85291130F2000C30F3002A08BA
:1002A000F000F1017208F00773080318013FF1072D
:1002B0007008C7007108C9000A08C8008A152B24F5
:1002C0008A11F00048088A007008CF0005308316B4
:1002D000C7000530C8007008C9008A156F228A114E
:1002E0004130FB00FF30FA00FB0B77297A29FA0B2B
:1002F00077297429C330FA00FA0B7C2900002A08F8
:10030000073A03198529AA0A47290330E9000B3067
:10031000EA008A15FA218A110530E9000530EA0061
:100320008A1565238A1105308316C7000530C80079
:100330005530C9008A156F228A11AA012A08073C84
:10034000031CDC29FF30F2000B30F3002A08F00018
:10035000F1017208F00773080318013FF1077008F4
:10036000C7007108C9000A08C8008A152B248A1121
:10037000F00048088A007008CF0005308316C700D7
:100380000530C8007008C9008A156F228A114130F3
:10039000FB00FF30FA00FB0BCE29D129FA0BCE2946
:1003A000CB29C330FA00FA0BD32900002A08073AF8
:1003B0000319DC29AA0A9E290430E9000B30EA005F
:1003C0008A15FA218A114E08013A031DF5294D0AB2
:1003D000F2007208CD007208783A031DF3298611E5
:1003E000CE01CD01F4298615F62986110030051AB3
:1003F0000130F2007208003A031D352A0130CE00A8
:1004000086151A30FC00FF30FB00FF30FA00FC0BB1
:100410000A2A112AFB0B0D2A102AFA0B0D2A0A2A86
:10042000072A7F30FB00FF30FA00FB0B182A1B2A3B
:10043000FA0B182A152A5830FA00FA0B1D2A000068
:1004400000000030051A0130F2007208003A031D66
:10045000342A0130D0000C30D10001308316CF0097
:100460008A1533218A11362AD62DD62D50088316A7
:10047000C700831251088316C8003E30C9008A1590
:1004800030238A110D30FC00FF30FB00FF30FA00F2
:10049000FC0B4B2A522AFB0B4E2A512AFA0B4E2AEE
:1004A0004B2A482ABF30FB00FF30FA00FB0B592AC9
:1004B0005C2AFA0B592A562A2B30FA00FA0B5E2ACC
:1004C0000000000000000130E9000130EA002030A7
:1004D0008316AB002030AC004130AD006C30AE0074
:1004E0006130AF007230B0006D30B100B201AB309E
:1004F0008312EB008A15B1228A114C08EE005230AB
:10050000EF008A15F2228A1101308312E9000C30C3
:10051000EA005230EB008A15B1228A1101308316AD
:10052000C7000F30C800B230C9008A1530238A11C5
:1005300001308316C7001030C8004330C9008A1547
:1005400030238A110230E9000130EA00203083169E
:10055000AB002030AC005230AD006130AE007A30DC
:10056000AF006C30B0006930B1006B30B200613068
:10057000B300B401AB308312EB008A15B1228A11AB
:100580004A08EE005D30EF008A15F2228A1102302F
:100590008312E9000C30EA005D30EB008A15B122CD
:1005A0008A1102308316C7000F30C800B230C9006C
:1005B0008A1530238A1102308316C7001030C80014
:1005C0004330C9008A1530238A110330E900013015
:1005D000EA0020308316AB002030AC005630AD006E
:1005E0006B30AE006C30AF006F30B0007030B100D7
:1005F000B201AB308312EB008A15B1228A114B088D
:10060000EE00A030EF008A15F2228A110330831227
:10061000E9000C30EA00A030EB008A15B1228A1103
:1006200003308316C7000F30C800B230C9008A15E6
:1006300030238A1103308316C7001030C8004330BE
:10064000C9008A1530238A110430E9000130EA001C
:1006500020308316AB002030AC005330AD00683042
:10066000AE007230AF006130B0006E30B100693062
:10067000B2002030B3002030B4002030B50020306C
:10068000B6004430B7004130B8002030B900203007
:10069000BA004E30BB004530BC00BD01AB30831208
:1006A000EB008A15B1228A110030051A0130F200E0
:1006B0007208003A031D5D2B812B00308518013034
:1006C000F2007208003A031D662BDD2B0130050590
:1006D000F2007208003A031D6E2B042C00308519BD
:1006E0000130F2007208003A031D772B262C0030EF
:1006F00005190130F2007208003A031D802B502CBE
:10070000362A5008043AFF30031D0030F200510829
:100710000C3AFF30031D0030F0007208F005031999
:10072000922B7A2C5008043AFF30031D0030F2005F
:100730005108103AFF30031D0030F0007208F00538
:100740000319A32B04285008033AFF30031D00307F
:10075000F20051080C3AFF30031D0030F00072081F
:10076000F0050319B62B0330E800C02C5008023AFC
:10077000FF30031D0030F20051080C3AFF30031D1A
:100780000030F0007208F0050319C92B0230E800B0
:10079000C02C5008013AFF30031D0030F200510810
:1007A0000C3AFF30031D0030F0007208F005031909
:1007B000DC2B0130E800C02C362A5008013A031D1A
:1007C000E22B362A5108103A031DE72B362A50082F
:1007D0008316C700831251088316C8002030C90051
:1007E0008A1530238A115003F0007008D000700879
:1007F0008316C700831251088316C8003E30C90013
:100800008A1530238A11362A5008043A031D092C10
:10081000362A50088316C700831251088316C80071
:100820002030C9008A1530238A11500AF000700860
:10083000D00070088316C700831251088316C800C1
:100840003E30C9008A1530238A11362A5008043AEE
:10085000FF30031D0030F2005108103AFF30031D35
:100860000030F0007208F00503194F2C5008831671
:10087000C700831251088316C8002030C9008A15AA
:1008800030238A110C30D10050088316C7000C3079
:10089000C8003E30C9008A1530238A11362A362A0C
:1008A0005008043AFF30031D0030F20051080C3AA2
:1008B000FF30031D0030F0007208F0050319792C99
:1008C00050088316C700831251088316C8002030D1
:1008D000C9008A1530238A111030D10050088316C0
:1008E000C7001030C8003E30C9008A1530238A1175
:1008F000362A362AE9014C08EA008A158A238A1129
:10090000C330FB00FF30FA00FB0B872C8A2CFA0B5C
:10091000872C842C4B30FA00FA0B8C2C0000013011
:1009200003138312E9004A08EA008A158A238A1110
:10093000C330FB00FF30FA00FB0B9F2CA22CFA0BFC
:100940009F2C9C2C4B30FA00FA0BA42C0000023098
:1009500003138312E9004B08EA008A158A238A11DF
:10096000C330FB00FF30FA00FB0BB72CBA2CFA0B9C
:10097000B72CB42C4B30FA00FA0BBC2C0000042826
:100980000830FC00FF30FB00FF30FA00FC0BC92CE4
:10099000D02CFB0BCC2CCF2CFA0BCC2CC92CC62C7E
:1009A000A530FB00FF30FA00FB0BD72CDA2CFA0B3A
:1009B000D72CD42CE730FA00FA0BDC2C00000030E6
:1009C00003138312051A0130F2007208003A031D66
:1009D000122D1A30FC00FF30FB00FF30FA00FC0B38
:1009E000F22CF92CFB0BF52CF82CFA0BF52CF22C35
:1009F000EF2C7F30FB00FF30FA00FB0B002D032DA6
:100A0000FA0B002DFD2C5830FA00FA0B052D0000D2
:100A100000000030051A0130F2007208003A031D90
:100A2000122D362A003085180130F2007208003A83
:100A3000031D742D6808013A031D382D64304C02E3
:100A40000318372D4C0AF0007008CC007008EE0037
:100A50005230EF008A15F2228A1101308312E90028
:100A60000C30EA005230EB008A15B1228A11742D45
:100A70006808023A031D562D0A304A020318552D04
:100A80004A0AF0007008CA007008EE005D30EF00FE
:100A90008A15F2228A1102308312E9000C30EA0032
:100AA0005D30EB008A15B1228A11742D6808033A73
:100AB000031D742D50304B020318732D4B0AF000A8
:100AC0007008CB007008EE00A030EF008A15F2220B
:100AD0008A1103308312E9000C30EA00A030EB00E9
:100AE0008A15B1228A11742D01300505F2007208B1
:100AF000003A031DD52D6808013A031D992D4C08B5
:100B0000463C0318982D4C03F0007008CC00700888
:100B1000EE005230EF008A15F2228A110130831262
:100B2000E9000C30EA005230EB008A15B1228A113C
:100B3000D52D6808023A031DB72D4A08013C031859
:100B4000B62D4A03F0007008CA007008EE005D3050
:100B5000EF008A15F2228A1102308312E9000C306C
:100B6000EA005D30EB008A15B1228A11D52D6808A4
:100B7000033A031DD52D4B08193C0318D42D4B0304
:100B8000F0007008CB007008EE00A030EF008A156E
:100B9000F2228A1103308312E9000C30EA00A030FF
:100BA000EB008A15B1228A11D52DC02C4A083907CD
:100BB000F20072083802031CEB2D06144B30D200F1
:100BC0003330D3005F30D400D5004F30D6004E30E4
:100BD000D700D801F82D06104B30D2003330D300A7
:100BE0005F30D4004F30D5004630D600D700D80152
:100BF0000030061B0130F4007408003AFF30031D7A
:100C00000030F2004B083802FF30031C0030F000C7
:100C10007208F00503191A2E06154B30DD0031302D
:100C2000DE005F30DF00E0004F30E1004E30E200D8
:100C3000E301272E06114B30DD003130DE005F303E
:100C4000DF004F30E0004630E100E200E301003019
:100C5000061B0130F4007408003AFF30031D003019
:100C6000F2004B083802FF30031C0030F00070081F
:100C70007205F4000030061A0130F2007208003AE2
:100C8000FF30031D0030F00070087405F5000030DF
:100C9000061A0130F4007408003AFF30031D0030DA
:100CA000F20028303B02FF30031C0030F0007008D7
:100CB0007205F4000030061B0130F2007208013AA0
:100CC000FF30031D0030F0007408F0057508F004D3
:100CD00003198E2E4C083A0203187D2E86144B30D1
:100CE0008316A0003230A1005F30A200A3004F3075
:100CF000A4004E30A500A6018D2E8312861041302F
:100D00008316A0006C30A1006130A2007230A300F5
:100D10006D30A4002130A500A6019D2E83128610FF
:100D20004B308316A0003230A1005F30A2004F305C
:100D3000A3004630A400A500A6018030CF008A158C
:100D400033218A115D30EE002A27C0308316CF0090
:100D50008A1533218A11A030EE002A279430831699
:100D6000CF008A1533218A115230EE002A271A301B
:100D7000FC00FF30FB00FF30FA00FC0BC02EC72E3A
:100D8000FB0BC32EC62EFA0BC32EC02EBD2E7F30FA
:100D9000FB00FF30FA00FB0BCE2ED12EFA0BCE2E2D
:100DA000CB2E5830FA00FA0BD32E000000004B284F
:100DB000D82E03138316C70183126F08F100013088
:100DC000F00071080319E82EF00D7010FF3FE22EBD
:100DD00070088316C9007009CA00C8014808073C9A
:100DE000031C272F83126E08840083164A0880058F
:100DF00084174A0880058A1523248A118316490816
:100E0000800484138A1523248A1183164908000557
:100E1000F1007108003A03191A2F4808F100013057
:100E2000F00071080319182FF00D7010FF3F122FFA
:100E30007008C7048A1532248A118A1532248A114F
:100E400083164808073A0319272FC80AEE2E4708C9
:100E5000F000080003138312EF016F086E0784008F
:100E60000008F1007108003A0319412F6F086E075E
:100E7000840000088316CE008A15EC238A11EF0A3D
:100E80002D2F080003138312690803178D008316A2
:100E90008C130C1483120C080313EA006A08F00088
:100EA0000800FF3FFF3FFF3FFF3FFF3FFF3FFF3F88
:100EB000FF3FFF3FFF3FFF3FFF3FFF3FFF3FFF3F42
:100EC000FF3FFF3FFF3FFF3FFF3FFF3FFF3FFF3F32
:100ED000FF3FFF3FFF3FFF3FFF3FFF3FFF3FFF3F22
:100EE000FF3FFF3FFF3FFF3FFF3FFF3FFF3FFF3F12
:100EF000FF3FFF3FFF3FFF3FFF3FFF3FFF3FFF3F02
:100F0000FF3FFF3FFF3FFF3FFF3FFF3FFF3FFF3FF1
:100F1000FF3FFF3FFF3FFF3FFF3FFF3FFF3FFF3FE1
:100F2000FF3FFF3FFF3FFF3FFF3FFF3FFF3FFF3FD1
:100F3000FF3FFF3FFF3FFF3FFF3FFF3FFF3FFF3FC1
:100F4000FF3FFF3FFF3FFF3FFF3FFF3FFF3FFF3FB1
:100F5000FF3FFF3FFF3FFF3FFF3FFF3FFF3FFF3FA1
:100F6000FF3FFF3FFF3FFF3FFF3FFF3FFF3FFF3F91
:100F7000FF3FFF3FFF3FFF3FFF3FFF3FFF3FFF3F81
:100F8000FF3FFF3FFF3FFF3FFF3FFF3FFF3FFF3F71
:100F9000FF3FFF3FFF3FFF3FFF3FFF3FFF3FFF3F61
:100FA000FF3FFF3FFF3FFF3FFF3FFF3FFF3FFF3F51
:100FB000FF3FFF3FFF3FFF3FFF3FFF3FFF3FFF3F41
:100FC000FF3FFF3FFF3FFF3FFF3FFF3FFF3FFF3F31
:100FD000FF3FFF3FFF3FFF3FFF3FFF3FFF3FFF3F21
:100FE000FF3FFF3FFF3FFF3FFF3FFF3FFF3FFF3F11
:100FF000FF3FFF3FFF3FFF3FFF3FFF3FFF3FFF3F01
:10100000DB23DB23DB2383163F08F0000130F400F1
:10101000700803190F28F40D7410FF3F0928740895
:101020008312A40083164008F0000130F30070081A
:1010300003191E28F30D7310FF3F1828730883123D
:10104000A50083164108F0000130F2007008031972
:101050002D28F20D7210FF3F272872088312A60078
:1010600083164208F0000130F100700803193C2893
:10107000F10D7110FF3F362871088312A700831607
:101080004408F00001308312A200700803194C28B4
:10109000A20D2210FF3F462883164508F0000130BC
:1010A0008312A900700803195928A90D2910FF3FC0
:1010B000532883164608F00001308312A1007008FF
:1010C00003196628A10D2110FF3F602883163E08F2
:1010D0008312A300831643088312A00083163E08E0
:1010E000840073087404F0007208F0047108F004BE
:1010F000F009700880058417831225082404F00085
:101100002608F0042708F004F0097008800584130D
:101110002008840029082204F0002108F004F009C6
:1011200070088005841729082204F0002108F004C3
:10113000F009700880058413230884002608000441
:10114000F000270870048000200884002108800433
:101150002109F00070088005DB23210880042109A3
:10116000F00070088005DB23210880042109F000CD
:1011700070088005DB2323088400260880042709E3
:10118000F0007008800520088400210880042109EF
:10119000F00070088005DB23210880042109F1009C
:1011A00071088005230884002609F0007008800576
:1011B0002408800420088400210880047108800528
:1011C000DB23230884002409F00070088005270829
:1011D000800420088400210880042109F10071089E
:1011E0008005230884002709F00070088005200886
:1011F00084002108800471088005DB232108800415
:101200002109F00070088005230884002708800465
:10121000200884002108800470088005DB2323084F
:1012200084002709F0007008800520088400210848
:1012300080042109F1007108800523088400270833
:101240000004F0002608F0042508F00424087004C7
:101250008000200884002108800471088005DB23B9
:101260000130A8000800031383122008840021091C
:10127000F000700880052209F0007008800523083E
:10128000840025082404F0002608F0042708F00450
:10129000F0097008800500308316CF1B0130F10083
:1012A0007108013A031D572983122408800403138F
:1012B0008312003083164F1B0130F1007108013A90
:1012C000031D65298312250880040313831200304F
:1012D0008316CF1A0130F1007108013A031D7329FA
:1012E00083122608800403138312003083164F1ADA
:1012F0000130F1007108013A031D8129831227088A
:10130000800403138312200884002808013A031D77
:101310008E292209F0007008800590292208800497
:101320002108800423242109F00070088005220987
:10133000F000700880052308840025082404F000CC
:101340002608F0042708F004F00970088005003032
:101350008316CF190130F1007108013A031DB3293A
:1013600083122408800403138312003083164F195C
:101370000130F1007108013A031DC12983122508CB
:1013800080040313831200308316CF180130F1005C
:101390007108013A031DCF29831226088004031324
:1013A0008312013083164F05F1007108013A031DC5
:1013B000DC29831227088004031383122008840089
:1013C0002808013A031DE9292209F0007008800568
:1013D000EB29220880042108800423242109F0003D
:1013E000700880052808013A031DF829DB23F92934
:1013F00032240800053003138316C7000530C800E7
:10140000BE30C9006F22AA012A08083C031C222A08
:101410000530EE000530EF008A11D9268A157008D4
:101420008312AB002C30F1002A08F1077108840008
:1014300071088400700880002A08083A0319222ADB
:10144000AA0A042A2D08B5002D08003A031D332AE4
:1014500069088316C70083126A088316C8002B30F8
:10146000C90030233D2A69088316C70083126A0821
:101470008316C8002D30C90030232C08B500013078
:101480002C05F1007108003A031D492A3030B600DE
:101490004B2A3530B6002C08F100F10CF11371081D
:1014A000B5003730F0006908F00770088400700854
:1014B0008400710880003508EE003C30EF00F22215
:1014C0003C308312EE008A112A278A152C308316AD
:1014D000CE00EC2336088316CE00EC23080003135D
:1014E00083164808F1000130F000710803197C2AC6
:1014F000F00D7010FF3F762A7008CC007009CD0007
:10150000CA014A08073C031CAE2A4A08F0004908F1
:10151000CB0070080319902ACB0CCB13FF3F8A2A0B
:101520000130CB05470884004D08800584174D081D
:10153000800584134B08003A0319A22A84174C082B
:1015400080048413F623841783164C0880048413C4
:101550004A08073A0319AE2ACA0A812A32243224D9
:101560000800031383126908013A031DBA2A803068
:10157000E900D12A6908023A031DC12AC030E900F6
:10158000D12A6908033A031DC82A9430E900D12AF8
:101590006908043A031DCF2AD430E900D12A8030EB
:1015A000E9006A03F0006908F0077008E9007008B4
:1015B0008316CF003321A801EC016C086B0784006F
:1015C0000008F2007208003A0319EF2A6C086B0752
:1015D000840000088316CE00EC23EC0ADD2A0130DB
:1015E000A8000800013003138316C70083126E0899
:1015F000093C0318FD2A8316C70A031383168312B6
:101600006E08633C0318062B8316C70A0313831660
:1016100083126F08840020308000840A8000840ACE
:101620008000840A8001840383164708003C031865
:101630002F2B0A30F40083126E08F000CA237808BA
:10164000F00030307007800084030A30F4006E0828
:10165000F000CA237008EE008316C703142B08009D
:10166000031383164708013A031D392B8030C70046
:10167000502B4708023A031D402BC030C700502BA7
:101680004708033A031D472B9430C700502B4708E7
:10169000043A031D4E2BD430C700502B8030C700B6
:1016A00048084707F000F0037008C70001308312B4
:1016B000A80070088316CF003321A80183164908BB
:1016C000CF0033210130A8000800031383126A08F9
:1016D000F1000130F00071080319722BF00D701049
:1016E000FF3F6C2B7008EC00F0097008ED006908F2
:1016F00084007008800584176D088005B6236C0887
:1017000080048413F6236C080005EB00B6236B08F5
:10171000F00008000030031783168C180130F10028
:101720007108013A031D962B00008A2B03138312C4
:10173000690803178D0003136A0803178C008316CA
:101740008C130C150B0803138312EB008B1355300D
:10175000031783168D00AA308D008C140313831297
:101760006B088B00031783160C1108000430031359
:101770008312FB00FF30FA00FB0BBF2BC22BFA0BCE
:10178000BF2BBC2B3730FA00FA0BC42B0000000033
:101790000000080003138312F8010830FC00700DEC
:1017A000F80D7408F8020318D72BF8070310F00D92
:1017B000FC0BCF2B0800243003138312FB00FF30F7
:1017C000FA00FB0BE42BE72BFA0BE42BE12B9E300A
:1017D000FA00FA0BE92B080003138312A801831601
:1017E0004E08CF0033210130A800080081300313D8
:1017F0008312FA00FA0BFA2B0000000008001034E4
:101800005434193451340134083400340C34080091
:1018100010349B343C3451340134083400349D344A
:10182000080010348D34213451340134083400342C
:10183000E434080010340034F334503401340834F4
:10184000003416340800013003138312FA00FA0B37
:10185000272C000008000313831249088A00470858
:1018600082000800533003138312FA00FA0B362C5F
:101870000800FF3FFF3FFF3FFF3FFF3FFF3FFF3FAE
:104200005A0004002800FF00FF00FF00FF00FF002D
:10421000FF00FF00FF00FF00FF00FF00FF00FF00A6
:10422000FF00FF00FF00FF00FF00FF00FF00FF0096
:10423000FF00FF00FF00FF00FF00FF00FF00FF0086
:10424000FF00FF00FF00FF00FF00FF00FF00FF0076
:10425000FF00FF00FF00FF00FF00FF00FF00FF0066
:10426000FF00FF00FF00FF00FF00FF00FF00FF0056
:10427000FF00FF00FF00FF00FF00FF00FF00FF0046
:10428000FF00FF00FF00FF00FF00FF00FF00FF0036
:10429000FF00FF00FF00FF00FF00FF00FF00FF0026
:1042A000FF00FF00FF00FF00FF00FF00FF00FF0016
:1042B000FF00FF00FF00FF00FF00FF00FF00FF0006
:1042C000FF00FF00FF00FF00FF00FF00FF00FF00F6
:1042D000FF00FF00FF00FF00FF00FF00FF00FF00E6
:1042E000FF00FF00FF00FF00FF00FF00FF00FF00D6
:1042F000FF00FF00FF00FF00FF00FF00FF00FF00C6
:10430000FF00FF00FF00FF00FF00FF00FF00FF00B5
:10431000FF00FF00FF00FF00FF00FF00FF00FF00A5
:10432000FF00FF00FF00FF00FF00FF00FF00FF0095
:10433000FF00FF00FF00FF00FF00FF00FF00FF0085
:10434000FF00FF00FF00FF00FF00FF00FF00FF0075
:10435000FF00FF00FF00FF00FF00FF00FF00FF0065
:10436000FF00FF00FF00FF00FF00FF00FF00FF0055
:10437000FF00FF00FF00FF00FF00FF00FF00FF0045
:10438000FF00FF00FF00FF00FF00FF00FF00FF0035
:10439000FF00FF00FF00FF00FF00FF00FF00FF0025
:1043A000FF00FF00FF00FF00FF00FF00FF00FF0015
:1043B000FF00FF00FF00FF00FF00FF00FF00FF0005
:1043C000FF00FF00FF00FF00FF00FF00FF00FF00F5
:1043D000FF00FF00FF00FF00FF00FF00FF00FF00E5
:1043E000FF00FF00FF00FF00FF00FF00FF00FF00D5
:1043F000FF00FF00FF00FF00FF00FF00FF00FF00C5
:02400E003A3F37
:00000001FF
